******************************************************************************
                  TI ARM Linker PC v5.1.1                      
******************************************************************************
>> Linked Mon Oct 13 13:26:44 2014

OUTPUT FILE NAME:   <TM4C129_I2CFIFO.out>
ENTRY POINT SYMBOL: "_c_int00"  address: 00000db9


MEMORY CONFIGURATION

         name            origin    length      used     unused   attr    fill
----------------------  --------  ---------  --------  --------  ----  --------
  FLASH                 00000000   00100000  00001329  000fecd7  R  X
  SRAM                  20000000   00040000  0000011c  0003fee4  RW X


SEGMENT ALLOCATION MAP

run origin  load origin   length   init length attrs members
----------  ----------- ---------- ----------- ----- -------
00000000    00000000    00001330   00001330    r-x
  00000000    00000000    00000200   00000200    r-- .intvecs
  00000200    00000200    00000e82   00000e82    r-x .text
  00001084    00001084    00000287   00000287    r-- .const
  00001310    00001310    00000020   00000020    r-- .cinit
20000000    20000000    0000011c   00000000    rw-
  20000000    20000000    00000100   00000000    rw- .stack
  20000100    20000100    0000001c   00000000    rw- .data


SECTION ALLOCATION MAP

 output                                  attributes/
section   page    origin      length       input sections
--------  ----  ----------  ----------   ----------------
.intvecs   0    00000000    00000200     
                  00000000    00000200     startup_ccs.obj (.intvecs)

.init_array 
*          0    00000000    00000000     UNINITIALIZED

.text      0    00000200    00000e82     
                  00000200    0000030c     uartstdio.obj (.text:UARTvprintf)
                  0000050c    00000204     driverlib.lib : sysctl.obj (.text:SysCtlClockFreqSet)
                  00000710    0000017c     TM4C129_I2CFIFO.obj (.text:main)
                  0000088c    00000130     driverlib.lib : gpio.obj (.text:GPIOPadConfigSet)
                  000009bc    0000009c     rtsv7M4_T_le_v4SPD16_eabi.lib : memcpy_t2.obj (.text)
                  00000a58    00000094                                   : auto_init.obj (.text)
                  00000aec    00000078                                   : memset_t2.obj (.text)
                  00000b64    00000074     uartstdio.obj (.text:UARTStdioConfig)
                  00000bd8    0000005e     rtsv7M4_T_le_v4SPD16_eabi.lib : copy_decompress_rle.obj (.text)
                  00000c36    00000002     startup_ccs.obj (.text:FaultISR)
                  00000c38    0000005c     uartstdio.obj (.text:UARTwrite)
                  00000c94    0000004c     TM4C129_I2CFIFO.obj (.text:ConfigureUART)
                  00000ce0    00000048     driverlib.lib : gpio.obj (.text:GPIOPinConfigure)
                  00000d28    00000048                   : i2c.obj (.text:I2CMasterInitExpClk)
                  00000d70    00000048                   : sysctl.obj (.text:_SysCtlFrequencyGet)
                  00000db8    00000048     rtsv7M4_T_le_v4SPD16_eabi.lib : boot.obj (.text)
                  00000e00    00000044                                   : cpy_tbl.obj (.text)
                  00000e44    00000044                                   : exit.obj (.text)
                  00000e88    00000042                                   : u_divt2.obj (.text)
                  00000eca    00000002     startup_ccs.obj (.text:IntDefaultHandler)
                  00000ecc    00000034     driverlib.lib : sysctl.obj (.text:SysCtlPeripheralEnable)
                  00000f00    0000002a                   : gpio.obj (.text:GPIODirModeSet)
                  00000f2a    00000024     uartstdio.obj (.text:UARTprintf)
                  00000f4e    00000002     startup_ccs.obj (.text:NmiSR)
                  00000f50    0000001c     driverlib.lib : sysctl.obj (.text:_SysCtlMemTimingGet)
                  00000f6c    00000018                   : i2c.obj (.text:I2CRxFIFOConfigSet)
                  00000f84    00000018                   : i2c.obj (.text:I2CTxFIFOConfigSet)
                  00000f9c    00000018     rtsv7M4_T_le_v4SPD16_eabi.lib : args_main.obj (.text)
                  00000fb4    00000014                                   : _lock.obj (.text)
                  00000fc8    00000012     driverlib.lib : gpio.obj (.text:GPIOPinTypeI2C)
                  00000fda    00000012                   : gpio.obj (.text:GPIOPinTypeI2CSCL)
                  00000fec    00000012                   : gpio.obj (.text:GPIOPinTypeUART)
                  00000ffe    0000000e                   : i2c.obj (.text:I2CFIFODataGet)
                  0000100c    0000000e                   : i2c.obj (.text:I2CFIFODataPut)
                  0000101a    0000000e                   : i2c.obj (.text:I2CRxFIFOFlush)
                  00001028    0000000e                   : i2c.obj (.text:I2CTxFIFOFlush)
                  00001036    0000000e     rtsv7M4_T_le_v4SPD16_eabi.lib : copy_decompress_none.obj (.text:decompress:none)
                  00001044    0000000a     driverlib.lib : i2c.obj (.text:I2CMasterEnable)
                  0000104e    00000008                   : i2c.obj (.text:I2CMasterBusy)
                  00001056    00000008                   : i2c.obj (.text:I2CMasterSlaveAddrSet)
                  0000105e    00000006     startup_ccs.obj (.text:ResetISR)
                  00001064    00000006     driverlib.lib : sysctl.obj (.text:SysCtlDelay)
                  0000106a    00000006                   : uart.obj (.text:UARTClockSourceSet)
                  00001070    00000006     rtsv7M4_T_le_v4SPD16_eabi.lib : copy_decompress_rle.obj (.text:decompress:rle24)
                  00001076    00000004     driverlib.lib : i2c.obj (.text:I2CMasterBurstLengthSet)
                  0000107a    00000004                   : i2c.obj (.text:I2CMasterControl)
                  0000107e    00000004                   : i2c.obj (.text:I2CMasterDataPut)

.const     0    00001084    00000287     
                  00001084    00000120     driverlib.lib : sysctl.obj (.const:g_pppui32XTALtoVCO)
                  000011a4    00000090                   : gpio.obj (.const:g_pui32GPIOBaseAddrs)
                  00001234    0000006c                   : sysctl.obj (.const:g_pui32Xtals)
                  000012a0    00000030                   : sysctl.obj (.const:g_sXTALtoMEMTIM)
                  000012d0    0000001c     uartstdio.obj (.const)
                  000012ec    00000012     uartstdio.obj (.const:.string)
                  000012fe    00000002     --HOLE-- [fill = 0]
                  00001300    00000008     driverlib.lib : sysctl.obj (.const)
                  00001308    00000003     TM4C129_I2CFIFO.obj (.const:.string)

.cinit     0    00001310    00000020     
                  00001310    0000000f     (.cinit..data.load) [load image, compression = rle]
                  0000131f    00000001     --HOLE-- [fill = 0]
                  00001320    00000008     (__TI_handler_table)
                  00001328    00000008     (__TI_cinit_table)

.stack     0    20000000    00000100     UNINITIALIZED
                  20000000    00000100     --HOLE--

.data      0    20000100    0000001c     UNINITIALIZED
                  20000100    00000008     rtsv7M4_T_le_v4SPD16_eabi.lib : _lock.obj (.data)
                  20000108    00000008                                   : exit.obj (.data)
                  20000110    00000005     uartstdio.obj (.data)
                  20000115    00000003     --HOLE--
                  20000118    00000004     rtsv7M4_T_le_v4SPD16_eabi.lib : stkdepth_vars.obj (.data)


LINKER GENERATED COPY TABLES

__TI_cinit_table @ 00001328 records: 1, size/record: 8, table size: 8
	.data: load addr=00001310, load size=0000000f bytes, run addr=20000100, run size=0000001c bytes, compression=rle


LINKER GENERATED HANDLER TABLE

__TI_handler_table @ 00001320 records: 2, size/record: 4, table size: 8
	index: 0, handler: __TI_decompress_rle24
	index: 1, handler: __TI_decompress_none


GLOBAL SYMBOLS: SORTED ALPHABETICALLY BY Name 

address    name
--------   ----
00000e45   C$$EXIT
00000c95   ConfigureUART
00000f01   GPIODirModeSet
0000088d   GPIOPadConfigSet
00000ce1   GPIOPinConfigure
00000fc9   GPIOPinTypeI2C
00000fdb   GPIOPinTypeI2CSCL
00000fed   GPIOPinTypeUART
00000fff   I2CFIFODataGet
0000100d   I2CFIFODataPut
00001077   I2CMasterBurstLengthSet
0000104f   I2CMasterBusy
0000107b   I2CMasterControl
0000107f   I2CMasterDataPut
00001045   I2CMasterEnable
00000d29   I2CMasterInitExpClk
00001057   I2CMasterSlaveAddrSet
00000f6d   I2CRxFIFOConfigSet
0000101b   I2CRxFIFOFlush
00000f85   I2CTxFIFOConfigSet
00001029   I2CTxFIFOFlush
0000105f   ResetISR
UNDEFED    SHT$$INIT_ARRAY$$Base
UNDEFED    SHT$$INIT_ARRAY$$Limit
0000050d   SysCtlClockFreqSet
00001065   SysCtlDelay
00000ecd   SysCtlPeripheralEnable
0000106b   UARTClockSourceSet
00000b65   UARTStdioConfig
00000f2b   UARTprintf
00000201   UARTvprintf
00000c39   UARTwrite
20000100   __STACK_END
00000100   __STACK_SIZE
20000100   __STACK_TOP
00001328   __TI_CINIT_Base
00001330   __TI_CINIT_Limit
00001320   __TI_Handler_Table_Base
00001328   __TI_Handler_Table_Limit
00000001   __TI_args_main
00000a59   __TI_auto_init
20000108   __TI_cleanup_ptr
00001037   __TI_decompress_none
00001071   __TI_decompress_rle24
2000010c   __TI_dtors_ptr
00000000   __TI_static_base__
00000aed   __aeabi_memclr
00000aed   __aeabi_memclr4
00000aed   __aeabi_memclr8
000009bd   __aeabi_memcpy
000009bd   __aeabi_memcpy4
000009bd   __aeabi_memcpy8
00000aef   __aeabi_memset
00000aef   __aeabi_memset4
00000aef   __aeabi_memset8
00000e89   __aeabi_uidivmod
ffffffff   __binit__
ffffffff   __c_args__
20000000   __stack
00000f9d   _args_main
00000db9   _c_int00
20000100   _lock
00000fc3   _nop
00000fbb   _register_lock
00000fb5   _register_unlock
20000104   _unlock
00000e49   abort
ffffffff   binit
00000e01   copy_in
00000e51   exit
00000000   g_pfnVectors
00000711   main
20000118   main_func_sp
000009bd   memcpy
00000af5   memset


GLOBAL SYMBOLS: SORTED BY Symbol Address 

address    name
--------   ----
00000000   __TI_static_base__
00000000   g_pfnVectors
00000001   __TI_args_main
00000100   __STACK_SIZE
00000201   UARTvprintf
0000050d   SysCtlClockFreqSet
00000711   main
0000088d   GPIOPadConfigSet
000009bd   __aeabi_memcpy
000009bd   __aeabi_memcpy4
000009bd   __aeabi_memcpy8
000009bd   memcpy
00000a59   __TI_auto_init
00000aed   __aeabi_memclr
00000aed   __aeabi_memclr4
00000aed   __aeabi_memclr8
00000aef   __aeabi_memset
00000aef   __aeabi_memset4
00000aef   __aeabi_memset8
00000af5   memset
00000b65   UARTStdioConfig
00000c39   UARTwrite
00000c95   ConfigureUART
00000ce1   GPIOPinConfigure
00000d29   I2CMasterInitExpClk
00000db9   _c_int00
00000e01   copy_in
00000e45   C$$EXIT
00000e49   abort
00000e51   exit
00000e89   __aeabi_uidivmod
00000ecd   SysCtlPeripheralEnable
00000f01   GPIODirModeSet
00000f2b   UARTprintf
00000f6d   I2CRxFIFOConfigSet
00000f85   I2CTxFIFOConfigSet
00000f9d   _args_main
00000fb5   _register_unlock
00000fbb   _register_lock
00000fc3   _nop
00000fc9   GPIOPinTypeI2C
00000fdb   GPIOPinTypeI2CSCL
00000fed   GPIOPinTypeUART
00000fff   I2CFIFODataGet
0000100d   I2CFIFODataPut
0000101b   I2CRxFIFOFlush
00001029   I2CTxFIFOFlush
00001037   __TI_decompress_none
00001045   I2CMasterEnable
0000104f   I2CMasterBusy
00001057   I2CMasterSlaveAddrSet
0000105f   ResetISR
00001065   SysCtlDelay
0000106b   UARTClockSourceSet
00001071   __TI_decompress_rle24
00001077   I2CMasterBurstLengthSet
0000107b   I2CMasterControl
0000107f   I2CMasterDataPut
00001320   __TI_Handler_Table_Base
00001328   __TI_CINIT_Base
00001328   __TI_Handler_Table_Limit
00001330   __TI_CINIT_Limit
20000000   __stack
20000100   __STACK_END
20000100   __STACK_TOP
20000100   _lock
20000104   _unlock
20000108   __TI_cleanup_ptr
2000010c   __TI_dtors_ptr
20000118   main_func_sp
ffffffff   __binit__
ffffffff   __c_args__
ffffffff   binit
UNDEFED    SHT$$INIT_ARRAY$$Base
UNDEFED    SHT$$INIT_ARRAY$$Limit

[75 symbols]
